:100000000C94D2010C94EF010C94EF010C94EF01CD
:100010000C94EF010C94EF010C94EF010C94EF01A0
:100020000C94EF010C94EF010C9490220C94622339
:100030000C94821D0C94EF010C94EF010C94EF01D1
:100040000C94EF010C94EF010C94EF010C94EF0170
:100050000C94EF010C940A1E0C94EF010C94EF0128
:100060000C94EF010C94EF010C94EF010C94EF0150
:100070000C94EF010C94EF010C94EF010C94EF0140
:100080000C94EF010C94EF010C94EF010C94EF0130
:100090000C94EF010C94EF010C94EF010C94EF0120
:1000A0000C94EF010C94EF010C94EF01C504C5040E
:1000B000F104F104590577058F068F0682051B06AA
:1000C0002C062C06CF23F623EE24F623EE2442241E
:1000D0006524EE24BC24CB244B004A0052004D0082
:1000E0004E00500051004F000251A900AE00AC007C
:1000F0000151AA00A800AB0029005F006000610068
:100100002B005C005D005E00280059005A005B0077
:100110000100620062003700C35CC65CC85CCA5C58
:10012000C45CC75CC95CCB5C010001000100005CE1
:10013000C15C010001000100000101010101010198
:10014000010102020202020202020203030303038C
:10015000030303040404040404040505050505065B
:100160000606060607070707070808080809090919
:10017000090A0A0A0B0B0B0C0C0C0D0D0D0E0E0EC2
:100180000F0F0F1010111111121213131414151553
:1001900016161717181819191A1A1B1B1C1D1D1EC5
:1001A0001E1F202021222223242425262627282919
:1001B000292A2B2C2D2D2E2F303132323334353647
:1001C0003738393A3B3C3D3E3F4041424344454647
:1001D0004748494A4C4D4E4F505153545556585923
:1001E0005A5B5D5E5F616264656668696B6C6D6FCA
:1001F0007072737577787A7B7D7E8082838587883D
:100200008A8C8E8F91939596989A9C9EA0A2A3A576
:10021000A7A9ABADAFB1B3B5B7BABCBEC0C2C4C677
:10022000C9CBCDCFD1D4D6D8DBDDDFE2E4E7E9EB33
:10023000EEF0F3F5F8FAFDFF1203430068006F00DB
:1002400063006F0070006100640000000E034B004B
:1002500065006500620069006F0000000403090486
:1002600009023B00020100A0FA0904000001030199
:100270000100092111010001224000070581030846
:10028000000109040100010300000009211101001F
:100290000122B600070582032000011201000200BE
:1002A00000000810CB441100010102000105010902
:1002B00002A10185020901A10005091901290815FA
:1002C00000250195087501810205010930093115E4
:1002D00081257F95027508810609381581257F954E
:1002E0000175088106050C0A38021581257F9501E4
:1002F00075088106C0C005010980A10185031901A7
:100300002AB700150126B700950175108100C005B8
:100310000C0901A101850419012AA002150126A0DA
:1003200002950175108100C005010906A10185062D
:10033000050719E029E715002501950875018102D7
:100340000507190029EF1500250195F075018102B7
:100350000508190129059505750191029501750397
:100360009101C005010906A101050719E029E7155A
:100370000025019508750181029501750881010527
:1003800007190029FF150026FF0095067508810052
:100390000508190129059505750191029501750357
:1003A0009101C00011241FBECFEFDAE0DEBFCDBF48
:1003B00011E0A0E0B1E0E6EEFBE402C005900D9292
:1003C000AA38B107D9F722E0AAE8B1E001C01D922E
:1003D000AA39B207E1F70E944A120C94F1250C9455
:1003E00000000E94481885E00E94B6180E940F176E
:1003F0004FEF6FEF80E00E94D51660E070E0CB0118
:100400000E94840D0C94900D81E0089581E0089580
:100410000C94060208950C940A021F93CF93DF9365
:1004200000D000D01F92CDB7DEB749835A836B83CB
:1004300030918D0189819A81311114C0662359F060
:10044000222349F00E94CA08182F682F89819A81B7
:100450000E94750803C00E949F08182F69817A8145
:10046000812F04C00E94CA0869817A810F900F9081
:100470000F900F900F90DF91CF911F910C94E60F8A
:10048000FC01262F408151816281738184810C940B
:100490000D0281E00895CF93DF93EC0160E00E94AC
:1004A0004002BE01DF91CF910C940B020C9413110A
:1004B0000C940F1108950E941F070E945A022FEFFB
:1004C00084E39CE0215080409040E1F700C00000B0
:1004D0000C94301E0F931F93CF93DF938C0161E038
:1004E0000E944002EC01B8010E940802882309F42E
:1004F0004BC0B801CE010E94BC18882309F444C047
:10050000B801CE010E94CE1B8823F1F1B801CE01C3
:100510000E94E2198823C1F1B801CE010E942A1B72
:10052000882391F1B801CE010E945817882361F108
:10053000F8018281882309F1CB358DE5D807C1F018
:1005400050F4C115FCE5DF0781F0CF3DDC45A9F48F
:100550000E94F40D19C0CC35EDE5DE0761F0CD3514
:10056000DD4559F40E94440D08C00E945B020CC096
:100570000E944D0D02C00E94500DC801DF91CF9125
:100580001F910F910C94040280E0DF91CF911F9195
:100590000F9108950E94651D80E00E94F1180C944F
:1005A000E8020E94E0170E94EB020C946B1D089574
:1005B0000C94D70281E008950C94DA020895CF9349
:1005C000C82F0E94D8028C2F0E94DC02CF91089580
:1005D00080E00C94DF020E942A1C0C94DF020E942F
:1005E0002A1C90918C01891721F080938C010C9426
:1005F000DF020895CF93DF93CDB7DEB72B970FB609
:10060000F894DEBF0FBECDBF4F83588769877A87C6
:100610008B8761110E94900C9E012F5F3F4F86E0F7
:10062000F90111928A95E9F785E0FE013796D90123
:1006300001900D928A95E1F789819A814C815D81C3
:10064000452B31F09F3F31F491E08F3F19F403C007
:1006500091E001C090E090FF09C049815A816B810F
:100660007C818D819E810E94B10B05C0C9010E94D1
:1006700049028111F2CF2B960FB6F894DEBF0FBE60
:10068000CDBFDF91CF910895FC01808191810E94BF
:100690000C090895CF93882309F4A4C0C82F823889
:1006A000C1F40E942A1C81FD9DC069E38091020172
:1006B000909103010E94201D0E94B20C2FEF81EE49
:1006C00094E0215080409040E1F700C0000069E3D1
:1006D00019C0833801F50E942A1C80FD83C063E5A0
:1006E00080910201909103010E94201D0E94B20C92
:1006F0002FEF81EE94E0215080409040E1F700C060
:10070000000063E580910201909103010E942B1D7E
:10071000CF910C94B20C8438C1F40E942A1C82FD43
:1007200061C067E480910201909103010E94201D45
:100730000E94B20C2FEF81EE94E021508040904057
:10074000E1F700C0000067E4DDCF8CEF8C0F813A49
:10075000D0F46C2F80910201909103010E94A01CA3
:10076000882349F06C2F80910201909103010E942F
:100770002B1D0E94B20C6C2F8091020190910301FD
:100780000E94201DC5CF80E28C0F883048F4C770CE
:1007900081E001C0880FCA95EAF70E94730CB8CFB8
:1007A000EBE5EC0FE33040F4F0E0E45BFE4F8081DA
:1007B00090E0CF910C945E1CE8E5EC0FE73150F42B
:1007C000F0E0EE0FFF1FE25EFE4F80819181CF913E
:1007D0000C94741CCD3E30F08C2F0E94CF12CF9120
:1007E0000C94A113CF910895882309F464C0823832
:1007F00079F40E942A1C81FF5EC069E380910201A6
:10080000909103010E94201D0E94B20C69E310C068
:100810008338B1F40E942A1C80FF4DC063E58091AB
:100820000201909103010E94201D0E94B20C63E519
:1008300080910201909103010E942B1D0C94B20C37
:10084000843879F40E942A1C82FF35C067E48091C5
:100850000201909103010E94201D0E94B20C67E4E6
:10086000E7CF9CEF980F913A10F4682FE1CF90E218
:10087000980F983050F4877091E001C0990F8A95D5
:10088000EAF7892F0E94790CD9CF9BE5980F933016
:1008900020F480E090E00C945E1C98E5980F97316E
:1008A00020F480E090E00C94741C8D3E20F00E94B7
:1008B0002A130C94A11308951F93CF93DF93182F3D
:1008C000EB010E944A03209741F08FE99FE00197D6
:1008D000F1F700C000002197F6CF812FDF91CF9173
:1008E0001F910C94F403893319F060E070E002C0AA
:1008F00060E570E00C945C04882321F00E94730C86
:100900000C94B20C0895882321F00E94790C0C9469
:10091000B20C0895CF92DF92EF92FF920F931F9344
:10092000CF93DF937C01D62FC72FFC011281058165
:1009300002950F700E94690C8823B9F01123A9F069
:100940008C2F807F803421F080E28D0F883068F01A
:1009500080916E0282FD09C082E00E94120D0E9409
:10096000690C91E0D82ED92601C0D12CCC2EC2948E
:100970008FE0C8228C2D90E08C30910508F0CFC11B
:10098000FC01EA5AFF4F0C947C258C2F807FCF709E
:10099000882311F0C295C07F112399F0CC2309F46C
:1009A000AAC180E28D0F883010F0D11104C08C2FC5
:1009B0000E94730C03C08C2F0E94830C0E94B20C07
:1009C0009AC18D2F0E94F403CC2309F4A8C180E2C0
:1009D0008D0F883038F1DD2329F18C2F0E94890C8E
:1009E00024C08C2F807FCF70803211F0C295C07FE1
:1009F000DD2319F0D130A1F13DC080916E0282FF5C
:100A000017C0112349F0CC2329F08C2F0E94730CBE
:100A10000E94B20C80E070C180E00E94F403CC23FD
:100A200009F47DC18C2F0E94790C0E94B20C77C111
:100A3000112371F0002341F0013031F40E94930C36
:100A40008C2B0E949B0C6BC10E94930C8C2B1DC0A5
:100A5000002319F0013009F462C10E94A80C25C0DE
:100A6000112321F0063008F05AC10EC0053008F0FD
:100A700056C11BC0112361F0002331F0F7018581BD
:100A800080FF39C18F7085838C2F0E947C0447C101
:100A9000002359F0D93309F03FC1FFEF07EE13E00F
:100AA000F15000401040E1F735C18C2F0E948304C3
:100AB00036C18C2F86958695837019F0813061F050
:100AC0002EC1112321F08D2F9C2F937002C080E046
:100AD00090E00E945E1C2BC1112321F08D2F9C2FD2
:100AE000937002C080E090E00E94741C20C18D2FA2
:100AF000112319F00E94CF1202C00E942A130E94F3
:100B0000A11315C18C2F837009F047C011110BC1BF
:100B10002D2F229526952770220F220F6D2F6F7093
:100B2000862F90E0A0E0B0E0022E04C0880F991F4D
:100B3000AA1FBB1F0A94D2F7D4FF10C04FE050E0A9
:100B400060E070E004C0440F551F661F771F2A95B0
:100B5000D2F7409550956095709503C040E050E005
:100B6000BA01C695C695C3708A019B01082B192B43
:100B70002A2B3B2BC901B801C23049F058F4C130CF
:100B800019F00E948B07CFC00E947907CCC00E9449
:100B90009D07C9C00E947707C6C0112319F08C2F8A
:100BA000817001C08695882309F4BDC02D2F229540
:100BB00026952770220F220F6D2F6F70862F90E0E1
:100BC000A0E0B0E0022E04C0880F991FAA1FBB1F2F
:100BD0000A94D2F7D4FF10C04FE050E060E070E01C
:100BE00004C0440F551F661F771F2A95D2F7409502
:100BF00050956095709503C040E050E0BA01C695ED
:100C0000C695C3708A019B01082B192B2A2B3B2BFD
:100C1000C901B801C23049F058F4C13019F00E943E
:100C2000500881C00E943E087EC00E9462087BC0BE
:100C30000E94B10778C0CF70112339F08C2F0E9429
:100C4000D7078D2F0E947C046EC08D2F0E948304D5
:100C50008C2F0E94F80767C0D23F21F128F4D03FC3
:100C600041F0D13FC1F043C0D33F19F1D43F79F0F7
:100C70003EC0112341F0053008F051C08C2F8F7118
:100C80000E941D084CC0063008F049C0F7CF809183
:100C90006E0282FF18C0112339F08C2F8F710E94D1
:100CA000D7073DC01123C9F38C2F8F710E94F8071D
:100CB00036C0112329F08C2F8F710E94C2072FC0DC
:100CC0000E94BD072CC0112349F0CF718C2F0E94C8
:100CD000D70763E08C2F0E94F70C21C081E00E94AF
:100CE000120D0230E0F082E00E94120D18C01123B4
:100CF00031F0002391F28D2F0E944A0310C000238F
:100D000099F2D93349F41FEF27EE33E01150204018
:100D10003040E1F700C000008D2F0E94F40388EFFF
:100D20008C0D843020F40E942A1C0E94DF02DD20FA
:100D3000C9F00E94650C80FD15C0F70112820E9467
:100D40005F0C0E94D707C7010E94D3060E945F0C68
:100D5000DF91CF911F910F91FF90EF90DF90CF9097
:100D60000C94F807DF91CF911F910F91FF90EF90B6
:100D7000DF90CF9008950F931F93CF93DF93EC01F3
:100D8000688179818A810E9417098C010E94740808
:100D90000E946507B801CE010E948A04DF91CF91BD
:100DA0001F910F910895CF93DF93EC019881898172
:100DB0002B813C81232B31F08F3F31F481E09F3F29
:100DC00019F403C081E001C080E080FD1DC0CE01A8
:100DD0000E946A02811110C00E94690C8823A1F050
:100DE0008A81882389F080916E0282FD0DC082E0A5
:100DF000DF91CF910C94120DCE010E94BB06CE0163
:100E0000DF91CF910C944B02DF91CF91089580E058
:100E100090E00E945E1C80E090E00E94741C0E94A2
:100E2000900C0E94B20C0E94D2140C94A1138091D9
:100E30000201909103010E94361D0C9407070E9445
:100E4000800C0C94170792959F70963079F010F4EF
:100E5000925001C09A50923068F4803F69F018F4C3
:100E6000883E40F409C0843F29F406C0883E20F043
:100E7000813F11F080E0089581E00895FC018081B8
:100E800091810E940C090E9423070895CF93DF935C
:100E900000D000D01F92CDB7DEB70F900F900F900B
:100EA0000F900F90DF91CF910895CF93DF9300D0F3
:100EB00000D000D0CDB7DEB726960FB6F894DEBFCF
:100EC0000FBECDBFDF91CF910895089508950C9482
:100ED00066070C9467070E94690760939C017093F2
:100EE0009D0180939E0190939F010C9407070C94A1
:100EF0006B070F931F9300919C0110919D0120910E
:100F00009E0130919F01602B712B822B932B1F919F
:100F10000F910C946B070F931F9300919C011091FC
:100F20009D0120919E0130919F01602371238223B6
:100F300093231F910F910C946B070F931F930091B4
:100F40009C0110919D0120919E0130919F0160278D
:100F50007127822793271F910F910C946B070C9494
:100F600066070E94AF076093980170939901809380
:100F70009A0190939B010C94070760E070E0CB010D
:100F80000C94B1070F931F9341E050E060E070E0D4
:100F90008A019B0104C0000F111F221F331F8A9575
:100FA000D2F7C901B8011F910F910C94B1070F93AB
:100FB0001F9341E050E060E070E004C0440F551F13
:100FC000661F771F8A95D2F78091980190919901B9
:100FD000A0919A01B0919B018A019B01082B192BCA
:100FE0002A2B3B2BC901B8011F910F910C94B1071B
:100FF0000F931F9341E050E060E070E004C0440FA5
:10100000551F661F771F8A95D2F7409550956095BA
:1010100070958091980190919901A0919A01B09159
:101020009B018A019B01082319232A233B23C90121
:10103000B8011F910F910C94B1070F931F9341E0DA
:1010400050E060E070E004C0440F551F661F771F3A
:101050008A95D2F78091980190919901A0919A0177
:10106000B0919B018A019B01082719272A273B275A
:10107000C901B8011F910F910C94B1070F931F93F1
:10108000009198011091990120919A0130919B0152
:10109000602B712B822B932B1F910F910C94B10716
:1010A0000F931F93009198011091990120919A013B
:1010B00030919B0160237123822393231F910F9111
:1010C0000C94B1070F931F9300919801109199010F
:1010D00020919A0130919B016027712782279327E5
:1010E0001F910F910C94B1070895990F990F890FD3
:1010F000E82FE695E695E695877051E001C0550F1B
:101100008A95EAF785E0E89FF0011124E257FE4F47
:1011100020E030E070E04081CB01022E02C09695C5
:1011200087950A94E2F78170819584278523842727
:1011300081932F5F3F4F2530310569F70895990F4F
:10114000990F890F682F669566956695982F977009
:1011500085E0689FB001112440E050E080E0FB0191
:10116000E40FF51FE257FE4F208130E0092E02C048
:10117000369527950A94E2F721703327042E01C093
:10118000220F0A94EAF7822B4F5F5F4F45305105DB
:1011900031F70895BF92CF92DF92EF92FF920F93B3
:1011A0001F93CF93DF938C01C0909801D090990149
:1011B000E0909A01F0909B0180919C0190919D019B
:1011C000A0919E01B0919F01C82AD92AEA2AFB2A40
:1011D000CFE1D0E0D701C6010C2E04C0B695A7958B
:1011E000979587950A94D2F780FD04C0219790F7D0
:1011F000B12C07C0BC2EB8018C2F0E94FA0F0197AA
:10120000A9F38B2DDF91CF911F910F91FF90EF905C
:10121000DF90CF90BF900895CF93DF93EC010E94B1
:10122000CA08BE010E94FA0FDF91CF9108951F9363
:10123000CF93DF93EB0190918D01992321F0CB01A6
:101240000E940C0913C0882349F0CB010E94CA08F0
:10125000182F682FCE010E94750804C0CB010E9490
:101260009F08182FBE01812F0E94FA0FDF91CF91A6
:101270001F9108951F93CF93DF93C091A00116E0B3
:101280008091A101C81799F0D0E01C9FF0011D9F2B
:10129000F00D1124EE55FE4F408151816281738122
:1012A000848195810E9455072196C770E9CFDF910F
:1012B000CF911F9108954091D2015091D301609137
:1012C000D4017091D5018091D6019091D7010C94F1
:1012D0005507EF92FF920F931F93CF93DF93809167
:1012E000D70182958F7009F065C08091D401882361
:1012F00009F460C08091A001F090A1011091D20189
:101300000091D3016091D5017091D60191E01F3F0A
:1013100009F090E0C0910001D0910101292F96E0E1
:10132000E92E8F1509F446C06115710521F00F3FB4
:1013300021F030E003C031E001C0322F90E030FDF9
:1013400036C0E89EF001E99EF00D1124DF01AE5594
:10135000BE4F11963C911197301329C03C91311327
:1013600026C012963C911297311121C013964D91CF
:101370005C911497461B570B4C175D07C0F4809186
:10138000D7018F7080618093D701E955FE4F80812E
:101390008F708061808382ED91E00E94D306DF919F
:1013A000CF911F910F91FF90EF900C943A09019605
:1013B0008770B7CFDF91CF911F910F91FF90EF9082
:1013C00008959F92AF92BF92CF92DF92EF92FF92D9
:1013D0000F931F93CF93DF93CDB7DEB761970FB60F
:1013E000F894DEBF0FBECDBF8C0185E0F801DE01B1
:1013F0001D9601900D928A95E1F7D8011296EC9016
:101400009091D201E091D3012091D5013091D60184
:101410002115310531F0EF3F31F481E09F3F19F4A0
:1014200003C081E001C080E0B82FB1709B2E80FD29
:1014300047C1D8014C9111965C9111971396AD90CC
:10144000BC90149782EDC82E81E0D82EF090D40184
:10145000B501621B730B2091000130910101FF2047
:1014600009F4D9C08091D7016217730708F095C0BD
:10147000282F207F09F052C05E1313C0491311C0FA
:10148000FE2CE1100EC08F7080618093D7010E9406
:101490005B09C6010E94D3068091D701F8018583BC
:1014A0004DC1AB2831F05F3F31F481E04F3F19F47B
:1014B00003C081E001C080E080FD03C081E08E2593
:1014C00002C080E090E0F82FF170FF2E80FF1CC07A
:1014D0008091A0012091A10136E0821709F40BC18F
:1014E00090E0389FF001399FF00D1124EE55FE4F2A
:1014F0006181561306C06081461303C06281E61203
:1015000003C001968770E9CFFE2CEE2009F416C1C6
:101510008091D70181608093D70154C05E1306C0CB
:10152000491304C0E11002C0F80199C0C8010E942B
:101530003E07882361F1EE2051F12091D701822FDF
:1015400082958F7090E0029774F08091D201909113
:10155000D30198878F831986BB86AA862C87CE01F4
:1015600007960E94D30686E0F801A2EDB1E0019053
:101570000D928A95E1F70E9469090E945B090AC0F1
:101580005E1711F1C8010E943E0781112CC0C801ED
:101590000E94D306FF24F394D1C0282F207F81F727
:1015A0007A2DB98AA88A6E2D89890E94460782ED14
:1015B00091E00E94D30686E0D6011D928A95E9F754
:1015C0000E945B09F12CBAC04913DCCFE110DACFDD
:1015D000F8018583C8010E94D30686E0D6011D92DA
:1015E0008A95E9F7ABC0EE2091F22091D701822FC6
:1015F00082958F7090E002970CF4B5CF8091D20164
:101600009091D3019A8389831B82BD82AC822E8301
:10161000CE010196A6CF6217730708F044C0FE2CD6
:10162000EE2009F4B4CF5E1330C049132EC02091D0
:10163000D70120FD21C0822F82958F70482F50E066
:1016400041155105C9F0F80125834F30510541F08E
:101650008F5F982F9295907F822F8F70892B858333
:10166000C8010E94D30686E0F801A2EDB1E0019026
:101670000D928A95E1F73CC086E0F801A2EDB1E059
:1016800001900D928A95E1F759C0C8010E943E076A
:10169000811169CF8091D70181608093D701C80102
:1016A0000E94D3064BC07A2DB98AA88A6E2D8989EB
:1016B0000E94460786E0D6011D928A95E9F718C078
:1016C000EE2009F464CFC8010E943E07F82E88235B
:1016D00009F45DCF86E0F801A2EDB1E001900D9232
:1016E0008A95E1F782ED91E00E9444030E94690926
:1016F0000E945B0923C04D875E878D859E850E9471
:101700000C09292F22952F70223028F49F7039F070
:10171000811105C00BC0243028F49F7049F4805E0D
:10172000883020F0C8010E94D3069F2CF92C06C0F7
:10173000D80115969C91907F91F7F8CF8F2D6196E7
:101740000FB6F894DEBF0FBECDBFDF91CF911F91D2
:101750000F91FF90EF90DF90CF90BF90AF909F9050
:1017600008951F93CF93DF93CDB7DEB72C970FB6B5
:10177000F894DEBF0FBECDBF4F83588769877A8745
:101780008B879C87CE0107960E94E1098823D1F0C0
:101790009F8188852A853B85232B31F08F3F31F44B
:1017A00081E09F3F19F403C081E001C080E080FD2B
:1017B00047C04F81588569857A858B859C850E94B5
:1017C00055073EC086E0FE013796DE011196019076
:1017D0000D928A95E1F7FF81E8856A857B85611521
:1017E000710531F0EF3F31F481E0FF3F19F403C0A0
:1017F00081E001C080E080FD23C02091A10130E0A4
:10180000C9010196877099274091A00150E0841783
:101810009507F1F1F983EA837D836C8396E0929FCB
:10182000D001939FB00D1124AE55BE4FFE013196ED
:1018300001900D929A95E1F78093A1010E943A09D7
:1018400016E08091A0019091A101891771F1189F74
:10185000C00111248E559E4F0E94E109882329F171
:10186000E091A0011E9FF0011124EE55FE4F408132
:10187000518162817381848195810E945507809195
:10188000A00190E00196877099278093A001D9CF9D
:101890000E941F071092A1011092A001E2EDF1E059
:1018A00086E0DF011D928A95E9F72C960FB6F89431
:1018B000DEBF0FBECDBFDF91CF911F910895809104
:1018C000F80185958595859508958091F801877033
:1018D00008959091F801977081E009F480E00895EF
:1018E00080911B02089590911B02892B80931B020B
:1018F0000895809590911B02892380931B0208957F
:1019000010921B02089590911A02892B80931A025B
:101910000895809590911A02892380931A02089560
:1019200010921A0208958091F901089508950C9477
:10193000960C0C94970C90916E0292FD08C09091B9
:10194000F901981721F08093F9010C94990C0895EE
:101950008091F901882329F01092F90180E00C941C
:10196000990C0895CF93DF93E0910201F091030168
:1019700080911B028083E0910201F091030190812C
:1019800080911A02892B80838091F901882381F04C
:10199000E0910201F09103019081892B8083809175
:1019A0000201909103010E948A1C81110E94A80CDF
:1019B000C0910201D091030140E250E068ED71E076
:1019C000CE010E949C25892B69F080E2FE01A8EDE2
:1019D000B1E001900D928A95E1F7CE01DF91CF91B0
:1019E0000C94361CDF91CF9108950C94960C909135
:1019F0006E0292FD10C098E0899F90011124262B61
:101A00002093F8010E94D7078091F801859585956C
:101A100085950C94F50C0C94D7071092F80180E092
:101A20000C94F50C2091F801809582238093F801A5
:101A3000982F977099F430E0482F082E000C550B22
:101A40002417350759F090916E0292FD07C08595D5
:101A5000859585950E94F8070C940D0D0895909139
:101A60006E0292FB222720F9281769F080FB92F979
:101A700090936E0280916D0290916E020E94770D9C
:101A800082E00C94120D089580916E0282FB8827EB
:101A900080F991E089270C942F0D81E00C942F0D93
:101AA00080E00C942F0D80E090E00E94B72521E0AB
:101AB000893E9E4F09F020E0822F089582E090E059
:101AC0000C94A92583E090E00C94A925CF9384E0A1
:101AD00090E00E94A925C82F82E290E00E94A925EB
:101AE0002C2F30E0A901582BCA01CF910895CF9334
:101AF000C92F682F84E090E00E94BD256C2F82E200
:101B000090E0CF910C94BD25AB01BC018FE090E03B
:101B10000C94CF25AB01BC0183E190E00C94CF2560
:101B200060E070E0CB010C948A0D69EE7EEF80E0FE
:101B300090E00E94DB2560E082E090E00E94BD25FD
:101B400060E083E090E00E94BD2510929C0110921D
:101B50009D0110929E0110929F0160E084E090E050
:101B60000E94BD2560E082E290E00E94BD2560E019
:101B700085E090E00E94BD2560E086E090E00E9454
:101B8000BD256FEF87E090E00E94BD2540E050E06A
:101B9000BA0188E090E00E94CF2560E08DE090E0FF
:101BA0000E94BD2540E050E0BA0188E190E00E942B
:101BB000CF2560E087E190E00E94BD2540E050E045
:101BC000BA018CE190E00E94CF2560E070E080E2F5
:101BD00090E00E94DB2540E050E0BA0188E190E00F
:101BE0000E94CF250C94F1010C94950D682F8EE086
:101BF00090E00C94BD250E94EF1D60932402709329
:101C0000250280932602909327026093200270930E
:101C100021028093220290932302089585B7806861
:101C200085BF85B7806885BF089581E008950C94CD
:101C3000150E08950C94190E0C94190E0C941C0E8C
:101C40000C94190E0C94200E0C94190E0E940E0E7A
:101C500086ED90E10E94201C0E94240E0C94220E1E
:101C60000E941A0E0C94190E0E94D9100E94DE02D6
:101C70000C94A7190E94DA1D0E94B0110E94340E24
:101C80000E94E0170E9421170C941E0E8F929F92C3
:101C9000AF92BF92CF92DF92EF92FF920F931F937A
:101CA000CF93DF93CDB7DEB72A970FB6F894DEBF98
:101CB0000FBECDBF0E94C511982E81110E94FB0D51
:101CC0008CE1A82E82E0B82E00E010E0802E802F5C
:101CD0000E94FD10D82EF501C1905F01C826B1F415
:101CE0000F5F1F4F0430110589F78FEF89838A83B7
:101CF0001B820E94E31D8160782F9D838C83498124
:101D00005A816B818D810E94FA022FC08091280236
:101D100081FD0E940311E12CFF24F3948C2D8F216F
:101D2000F1F00E94170E882399F0EE828F82DF2057
:101D300081E009F480E088870E94E31D8160782FAC
:101D40009A8789874E815F8168858A850E94FA0219
:101D5000F801E45EFD4F8081F826F08206C0E3942E
:101D6000FF0CF4E0EF12DACFBBCF81E0911001C09D
:101D700080E02A960FB6F894DEBF0FBECDBFDF918C
:101D8000CF911F910F91FF90EF90DF90CF90BF9078
:101D9000AF909F908F9008950E94460E0E94A619C2
:101DA0000E94BF130C94EF02CF93DF930E94FF0FAA
:101DB000EC01811521E5920708F045C0811530E559
:101DC000930708F094C0883E910528F5803E910560
:101DD00008F0F8C0883A910570F4853A910508F04A
:101DE0007CC08130910509F475C008F4E8C00497FF
:101DF00008F0E8C0E4C08F3B910508F0E0C0C85A85
:101E0000D0E0CC0FDD1FC15BDE4F0990D881C02D23
:101E1000CE019464D8C0811540E2940758F481152E
:101E200051E0950708F0CEC08D3E910508F4C7C07B
:101E30009065C9C0C11580E4D80708F4C0C0DF7040
:101E4000CE01906AC0C0811525E59207A8F48115DE
:101E500034E5930708F095C0811543E5940708F031
:101E60007BC0811552E5950708F061C0D82FCC27BB
:101E7000CE01816F906AA7C0C11589E5D807A0F48B
:101E8000C11528E5D20708F082C0C11536E5D30791
:101E900008F095C08C2F0E9493108F7190E0D82F7E
:101EA000CC27CE0190628FC0C1154AE5D40708F453
:101EB00074C0CE0190568115904208F080C08D2FDD
:101EC0008F710E949310DD27D0628F71AE01582B65
:101ED000CA0179C081E090E076C0C55AD0E0C3580D
:101EE000DE4F8881C82FD0E0CE0190646CC074E0D2
:101EF000969587957A95E1F7282F23703C2F3370BC
:101F000081E090E002C0880F991F3A95E2F79C6843
:101F1000AC01522B9A019C2F9F709695969550E29A
:101F2000959FE0011124C9018C2B9D2B4CC083701F
:101F3000992721E030E002C0220F331F8A95E2F793
:101F40009C2F9695969580E2989FE0011124C22BD4
:101F5000D32BCE019C6837C08370992721E030E0F5
:101F600002C0220F331F8A95E2F79C2F9695969513
:101F700040E2949FE0011124C22BD32BCE019A683A
:101F800022C0D82FCC27CE01846F906A1CC0DC2FD2
:101F9000CC27CE01806F906A16C08C2F8F700E9464
:101FA000931094E0D695C7959A95E1F7CF70D0E05D
:101FB000DC2FCC27D0699E01282BC90104C080E00A
:101FC00090E001C0CE01DF91CF910895E72FF0E0BE
:101FD00094E0899FE00DF11D1124EE0FFF1FEE0F1D
:101FE000FF1FE60FF11DEE0FFF1FE852FF4F859117
:101FF000949108950E94E60F0E94D40E08958238AD
:10200000910569F1B0F48133910509F46DC048F48C
:102010008932910509F463C08A32910509F469C0D7
:1020200008958533910509F455C089339105B9F0B8
:102030000895833E910569F138F4803E9105B1F031
:10204000823E910509F10895863E9105A9F1873EEA
:102050009105B9F1843E910509F064C023C0209137
:102060006D0220FD4FC021FD4DC0089580916D028D
:1020700080FD44C080916E0280FF44C080916D025B
:1020800084FD42C083EE4DC080916D0282FF38C056
:10209000F5CF80916D0282FD33C080916E0280FD8C
:1020A00031C0ECCF80916E0281FF32C080916D0211
:1020B00084FD2AC087EE35C080916D0283FF26C063
:1020C000F5CF80916D0283FD21C080916E0281FD6C
:1020D0001FC0ECCF80916D0285FD1CC01DC080919A
:1020E0006D0285FD19C016C080916D0286FD16C077
:1020F00017C080916D0286FD13C010C089E311C026
:1021000082EE0FC080EE0DC080E00BC086EE09C0ED
:1021100084EE07C089E205C085E303C08AE201C0FE
:1021200081E390E0089590916D0292FF0DC0282FF9
:102130002871283019F4877F846006C0282F247105
:10214000243011F48B7F886093FF0DC0282F2871F5
:10215000283119F4877E846106C0282F2471243128
:1021600011F48B7E886120916E0220FF0DC0382F04
:102170003871383019F4877F816006C0382F31718B
:10218000313011F48E7F886021FF0DC0282F287117
:10219000283119F4877E816106C0282F21712131F1
:1021A00011F48E7E886194FD877E089580E0089505
:1021B00008950E94530D811102C00E94F40D0E94E7
:1021C0005E0D809328020E94660D90936E028093AC
:1021D0006D020E94D8100E94620D682F70E080E0AE
:1021E00090E00E9477076091980170919901809129
:1021F0009A0190919B010C94AF07E82FF0E0ED5805
:10220000FD4F80810895089580EA8A95F1F7089539
:1022100000C008950C94041108950C940C110C94B2
:102220000D110C940C110C941111F894E82FE295F7
:10223000EF70F0E031A1282F2F7081E090E001C015
:10224000880F2A95EAF7982F9095932391A392A14E
:10225000892B82A3789408950F931F93CF93DF93D4
:10226000C4E8D1E089918F3F11F00E94151181E0FF
:10227000C838D807B9F7C0E8D1E004E811E089917F
:102280008F3F11F00E9415110C171D07C1F7DF9148
:10229000CF911F910F910895CF92DF92EF92FF920D
:1022A0000F931F93CF93DF938C01C62FD0E0CE0105
:1022B0008C579E4F7C01FC0190819F3F09F447C0E1
:1022C000D62EF894E92FE295EF70F0E081A19F708F
:1022D00021E030E001C0220F9A95EAF7822B81A31A
:1022E00082A12095282322A378940E940811E0E877
:1022F000F1E044E851E031E0C12C21912F3F89F019
:10230000A22FA295AF70B0E090968C9190E02F70C4
:1023100002C0959587952A95E2F780FD02C0832F2C
:1023200001C080E0C82A330F4E175F0731F7F7016D
:1023300080818F3F11F00E94151161E0C11001C032
:1023400060E08D2D0E940A11C00FD11FC882DF915D
:10235000CF911F910F91FF90EF90DF90CF90089554
:102360000E942C1184E0E3E7F2E0DF01982F1D9238
:102370009A95E9F7EFE6F2E0DF011D928A95E9F719
:1023800084E00E9407120C9456021F93CF93DF93B0
:1023900000D000D0CDB7DEB719821A821B821C8212
:1023A00010E0612FCE0101960E944C111F5F143086
:1023B000C1F744E050E0BE016F5F7F4F8FE692E0CF
:1023C0000E949C2511E0009709F410E0892B61F030
:1023D00089819A81AB81BC8180936F029093700256
:1023E000A0937102B0937202212F44E063E772E080
:1023F0008FE692E00E9408120E945802812F0F90EF
:102400000F900F900F90DF91CF911F910895089535
:10241000FF920F931F93CF93DF938C01F62ED72F4C
:10242000C42F222349F081E080932B020E94E31DF8
:1024300090932A028093290280912B028823C1F075
:102440008091290290912A020E94FB1D059780F03D
:10245000EF2DFD2FD8014C2F50E0CD01801B910BAB
:10246000841795071CF48D918193F7CF10922B025E
:10247000DF91CF911F910F91FF9008950E94E81F67
:102480000E943A0E0C94F41F0E94F81F0E94CC0E7A
:102490000C9412200E94811D0E94CF1F0E94260EC4
:1024A0000E943E120E9444120E94300EFBCF809187
:1024B000320280FF06C06091090170E0660F771F4D
:1024C00026C081FF04C06091090184E005C082FF3D
:1024D00007C06091090188E0689FB001112417C00E
:1024E000909131029923D1F060910801961788F7F5
:1024F0002091090188E0289F90011124929FA0015A
:10250000939F500D112470E0CA010E944625603847
:10251000710540F46115710519F406C068E070E0BA
:10252000862F08958FE7089581E008958091320203
:1025300080FF08C06091050170E0759567957595FD
:10254000679521C081FF06C06091050170E0759517
:10255000679519C082FF04C06091050170E010C04A
:1025600090913002992399F0609104019617A0F799
:1025700080910501899FC001112470E00E944625C9
:102580006038710540F46115710519F406C061E009
:1025900070E0862F08958FE7089581E008958D3EBD
:1025A00021F40E945712819504C08E3E29F40E94A6
:1025B00057128093360208958F3E21F40E945712DD
:1025C000819504C0803F29F40E9457128093350200
:1025D0000895893F19F40E94961205C08A3F31F48C
:1025E0000E94961281958093370208958B3F21F4C3
:1025F0000E949612819504C08C3F29F40E94961285
:102600008093380208959FE0980F983078F421E085
:1026100030E0A90102C0440F551F9A95E2F7CA01A4
:1026200090913402892B8093340208958D3F21F4D8
:102630008091320281600BC08E3F21F48091320282
:10264000826005C08F3F29F48091320284608093BC
:10265000320208958D3E39F49091360297FF35C0CD
:102660001092360259C08E3E29F490913602191606
:10267000BCF32BC0909135028F3E29F497FF25C003
:102680001092350249C0803F19F41916CCF31DC0D1
:1026900090913702893F29F41916BCF41092370241
:1026A0003BC08A3F19F497FF10C0F8CF8B3F39F435
:1026B0009091380297FF09C0109238022DC08C3FCC
:1026C00021F4909138021916BCF39FE0980F9830CE
:1026D00080F421E030E0A90102C0440F551F9A9513
:1026E000E2F7CA01809590913402892380933402E5
:1026F00013C08D3F21F4809132028E7F0BC08E3F3C
:1027000021F4809132028D7F05C08F3F29F48091A2
:1027100032028B7F8093320280913502811106C094
:1027200080913602811102C01092310280913702ED
:10273000811106C080913802811102C010923002CE
:1027400008950E94E31D20913502211104C02091BB
:102750003602222321F090932F0280932E022091A3
:102760003702211104C020913802222321F09093D6
:102770002D0280932C0283E392E00C94501CEF9284
:10278000FF920F931F93CF93DF9300D000D000D020
:10279000CDB7DEB786E0E3E3F2E0DE01119601900B
:1027A0000D928A95E1F7E0903502F09036020091A3
:1027B00037021091380210923502109236021092B0
:1027C000370210923802E11003C0FF2009F45DC007
:1027D00080912E0290912F020E94FB1DAC019091DE
:1027E0003102992339F020910A0130E0241735078E
:1027F00058F04BC020910B018AE0289F90011124D2
:102800002417350718F041C09F3F19F09F5F909340
:102810003102EE2061F00E9457121E1414F09FEF57
:1028200001C091E0989F902D112490933502FF20D4
:1028300061F00E9457121F1414F09FEF01C091E045
:10284000989F902D112490933602309135023323B6
:10285000E1F0209136022223C1F045EB3403C001A0
:102860001124992319F09093350203C081E08093DD
:10287000350235EB2303C0011124992319F09093FD
:10288000360203C081E080933602011103C0112398
:1028900009F45DC080912C0290912D020E94FB1DD5
:1028A000AC0190913002992339F02091060130E07B
:1028B0002417350758F04BC0209107018AE0289F64
:1028C000900111242417350718F041C09F3F19F0DB
:1028D0009F5F90933002002361F00E9496121016C1
:1028E00014F09FEF01C091E0989F902D11249093D8
:1028F0003702112361F00E949612111614F09FEF17
:1029000001C091E0989F902D11249093380230914E
:1029100037023323E1F0209138022223C1F045EB46
:102920003403C0011124992319F09093370203C096
:1029300081E08093370235EB2303C00111249923F2
:1029400019F09093380203C081E08093380280919F
:10295000350281110BC080913602811107C0809130
:102960003702811103C08091380281110E94A113A6
:10297000EB82FC820D831E8386E0FE013196A3E389
:10298000B2E001900D928A95E1F726960FB6F89481
:10299000DEBF0FBECDBFDF91CF911F910F91FF9092
:1029A000EF900895E3E3F2E086E0DF011D928A955F
:1029B000E9F710923102109230021092320208951B
:1029C000EF92FF920F931F93CF93DF938B01682FAA
:1029D00011110AC0442329F0E82FF0E0E85CFE4F13
:1029E0006491762F862F75C0212F30E0E82FF0E01C
:1029F000442321F0E85CFE4FE491F0E046E0049FC0
:102A0000C0011124CFEFD0E0BE010E9432254BEA75
:102A10004603C001479F900D1124800F911D800F28
:102A2000911D982F990F890FAE01421B530B4E9F9A
:102A3000D0014F9FB00D5E9FB00D11249B2F189FAA
:102A4000A0011124452F55278E01041B150B0E9F45
:102A5000A0010F9F500D1E9F500D11247E01E81AFA
:102A6000F108E29E8001E39E100DF29E100D1124EC
:102A7000212F3327C21BD30BCE9F9001CF9F300D48
:102A8000DE9F300D112462307105A9F048F4611504
:102A9000710569F061307105C9F48B2F752F0DC078
:102AA0006430710581F058F06630710579F47E2F3D
:102AB0008B2F932F0DC0832F7B2F9E2F09C08E2F1E
:102AC0007B2F952F05C08E2F732F02C07E2F852F51
:102AD000692FDF91CF911F910F91FF90EF90089593
:102AE00041E00E94E01408950E9470150895CF936C
:102AF000DF93762FE901682F842F0E947415798364
:102B000068838A83DF91CF91089580917702982F0F
:102B10009695913021F081708260809377020895BC
:102B200088E090E00C94B125CF92DF92EF92FF9273
:102B30006B017C010E948515B701A60188E090E039
:102B4000FF90EF90DF90CF900C94CF25E7E7F2E075
:102B500083E0808311828FEF82838383148260817C
:102B60007181828193810C94941590917B029330B2
:102B700018F49F5F90937B02882351F06091770255
:102B8000709178028091790290917A020C94941558
:102B9000089581E00C94B51590917B02992319F06A
:102BA000915090937B02882351F06091770270914D
:102BB00078028091790290917A020C94941508958C
:102BC00081E00C94CC1570E00C94B71960910D0164
:102BD0008091770280FF0AC080910C0123E0829FE0
:102BE000C001112484589D4F0C94E31580910E016F
:102BF00090910F01891780F7E82FF0E09F01220FD5
:102C0000331FE20FF31FE458FD4F1182108212822E
:102C10008F5FF0CFE7E7F2E080818E7F8083608175
:102C20007181828193810E9494152FEF80E792E059
:102C3000215080409040E1F700C000000C94E61560
:102C40009091770290FF16C090910E0120910F0194
:102C5000921770F4E92FF0E0DF01AA0FBB1FEA0F13
:102C6000FB1FE458FD4F8183608342839F5FF0CF59
:102C70000C94E6150895EF92FF920F931F93CF9354
:102C8000DF9300D01F92CDB7DEB79091770290FF0F
:102C90002CC0E22E142F062FF82EE92FE695F0E037
:102CA000E857FE4F808180933A029E7F923059F41C
:102CB0009E012F5F3F4F8F2D0E9477154B816981B9
:102CC0008A810E942016F092780200937902109374
:102CD0007A02EE2051F06091770270917802809133
:102CE000790290917A020E9494150F900F900F90A4
:102CF000DF91CF911F910F91FF90EF900895E7E73B
:102D0000F2E09181282F4381628188E0890F0C9441
:102D10003B1681E00C947F16E7E7F2E09181282FC3
:102D20004381628188EF890F0C943B1681E00C94FB
:102D30008C16E7E7F2E0628128E0620F08F46FEF9B
:102D4000282F438181810C943B1681E00C949916C5
:102D5000E7E7F2E0628128E0621B08F460E0282FD8
:102D6000438181810C943B1681E00C94A816E7E71F
:102D7000F2E0438128E0420F08F44FEF282F6281F0
:102D800081810C943B1681E00C94B716E7E7F2E0E2
:102D9000438128E0421B08F440E0282F62818181B2
:102DA0000C943B1681E00C94C61621E00C943B1663
:102DB00020E00C943B168091770280FF18C0817050
:102DC000826080937702662351F060917702709160
:102DD00078028091790290917A020E949415409134
:102DE0007A0260917902809178020C94D816089545
:102DF000682F81E00C94DB1681E00C94F816682FA4
:102E00009091770296958FEF890F09F481E00C94E9
:102E1000DB1681E00C94FF1661E00C94DB16E7E70B
:102E2000F2E080818160808386950C940C178091FC
:102E3000770280FD0C940A160C940F1760E00C9436
:102E4000DB168091390281112CC00E94530D811133
:102E500004C00E94F40D0E94A6150E949015609374
:102E60007702709378028093790290937A026E7F52
:102E700061F40E94A6150E949015609377027093EA
:102E800078028093790290937A020E94851580914E
:102E9000770280FF03C086950E941E1781E0809311
:102EA00039020895882311F0FA0101C0FB01099449
:102EB0001F93CF93DF93FB01128111116BC0EC01C3
:102EC0000E94700C8272CA3CFCE5DF0709F450C016
:102ED000C0F4C63CECE5DE07E1F148F4C43C9CE5F7
:102EE000D90759F178F5C33CDC4521F121C0C83C34
:102EF0009CE5D90799F1B8F549E856E166E976E12C
:102F000025C0CE3CFCE5DF0709F441C050F4CC3CC1
:102F1000ECE5DE0791F1B0F543EC56E162ED76E1C8
:102F200015C0C73D8CE5D807A8F1CE35DD4591F138
:102F300011E030C00E9417172DC049E057E16CEF37
:102F400076E104C04CEF56E169E077E10E94521748
:102F500021C046E956E169E876E1F8CF44EB56E155
:102F600065EA76E1F3CF45EA56E164EB76E1EECF30
:102F700042ED56E163EC76E1E9CF40EE55E169ECD4
:102F800075E1E4CF49EC55E160EE75E1DFCF81E01A
:102F90000E940C17812FDF91CF911F91089586E039
:102FA00090E00C94A925682F86E090E00C94BD2554
:102FB0008091880284708163809388020C94D31777
:102FC0000E94530D811104C00E94F40D0E94D81775
:102FD0000E94CF1780938802282F26952695269544
:102FE00030E02730310524F08770806380938802B9
:102FF0008091880280FF04C086958695869501C0E1
:1030000080E00C94F11820918802822F8695869595
:103010008695482F50E04630510554F48F5F982F25
:10302000990F990F990F822F8770892B80938802AF
:10303000809188028160809388020E94D3178091DA
:1030400088028695869586950C94F1188091880261
:10305000982F969596959695A1F0915E990F990F58
:10306000990F8770892B80938802887F91E009F4FB
:1030700090E08091880290FB80F9809388020E9402
:10308000D317809188028695869586950C94F118C1
:103090008091880280FD13C0816080938802813016
:1030A00019F489E080938802809188020E94D317E6
:1030B000809188028695869586950C94F1180895DE
:1030C0008091880280FF08C08E7F809388020E94D2
:1030D000D31780E00C94F11808958091880280FD48
:1030E0000C9460180C94481890918802892F86954A
:1030F000869586958F5F8F719770873038F4880F2B
:10310000880F880F892B8093880202C090938802D1
:1031100080918802887F91E009F490E08091880294
:1031200090FB80F9809388020E94D31780918802D7
:103130008695869586950C94F118873008F086E080
:10314000909188029770282F220F220F220F922B26
:1031500090938802987F21E009F420E09091880202
:1031600020FB90F9909388020C94F1180E949D180E
:10317000809188020C94D3179C01FB0182818823E3
:1031800049F12E3BFCE53F07C9F040F42C3BECE550
:103190003E0769F02D3B3C4561F00895203C9CE5DD
:1031A000390791F070F0213C3C4589F0089586E0A4
:1031B00001C080E00E94B61880E008950E942618A1
:1031C000FBCF0E940318F8CF0E946D18F5CF0E9424
:1031D0007418F2CF81E00895259A2D9808952D98BE
:1031E00008958F929F92AF92BF92CF92DF92EF920B
:1031F000FF920F931F93CF93DF93C82F873050F424
:10320000811109C0809180008F77809380000E9497
:10321000EF1806C0C6E0809180008068809380002F
:10322000A0918600B09187002C2F30E00E9482256B
:1032300026E030E040E050E00E945A250027122F9F
:10324000232F342F012F122F232F33278091860015
:10325000909187006CE070E00E9432256017710742
:1032600030F0C80169E070E00E9432255EC08091B4
:10327000860090918700E0908600F0908700E091B2
:103280008600F0918700C6E0D0E0BE010E943225A2
:10329000060F171F211D311D4801590185E0880CBB
:1032A000991CAA1CBB1C8A95D1F7C701BE010E94BC
:1032B00032256F01E12CF12CA7019601260F371F53
:1032C000411D511DC501B4010E945A2569017A01B1
:1032D000E0918600F0918700CA01B9010E94222581
:1032E0009B01AC01DF010E9491259B01AC01C7014C
:1032F000B6010E942225DC01CB012FE0B695A795EF
:10330000979587952A95D1F70091860010918700AF
:1033100020E030E0081719072A073B0728F46091DE
:10332000860070918700CB01BC0170938900609387
:103330008800DF91CF911F910F91FF90EF90DF9068
:10334000CF90BF90AF909F908F90089508950E9466
:10335000EC1882E88093800089E1809381008FEFF0
:103360009FEF90938700809386000C94E017539A08
:103370002BB1277F3BB138604FB7F894FC01CB01EC
:10338000880F991F680F791F6E0F7F1FE617F707C9
:1033900089F0819198E03BB9000000C087FF2BB90C
:1033A000880F000000C000C000C02BB900C09A9573
:1033B00091F7ECCF4FBF8FE594E00197F1F700C094
:1033C00000000895CF93DF93EC01FB0182818823F5
:1033D00009F43CC1C430FDE5DF0760F4CB3F9CE558
:1033E000D90788F49E0122503C452431310508F06C
:1033F0002EC109C0C236EDE5DE0729F0C63AFDE56B
:10340000DF0709F024C10E94660D90936E0280933D
:103410006D02C1318CE5D80709F4C6C008F042C07E
:10342000C930ECE5DE0709F49BC000F5C5308CE53A
:10343000D80709F485C078F4C330ECE5DE0709F459
:1034400078C008F07AC0C230DC4509F0F5C0809140
:103450006D028160EFC0C7309CE5D90709F478C0E0
:1034600008F07AC080916D028061E4C0CD30FCE547
:10347000DF0709F487C058F4CB309CE5D90709F47D
:1034800079C008F07BC080916D0288606FC0CF303A
:10349000FCE5DF0709F480C008F082C080916D026E
:1034A000877FC8C0CE3F9CE5D90709F471C000F5FD
:1034B000C531FCE5DF0709F485C068F4C3319CE53C
:1034C000D90709F475C008F095C00E941F078091C4
:1034D0006D028F77AFC0CC3FFCE5DF07A9F108F0A4
:1034E00054C0CB3FDC4509F0A7C080916E0240C0BC
:1034F000C230EDE5DE0709F489C058F4C1158DE549
:10350000D80709F45AC008F069C080916E02826041
:103510002FC0C236EDE5DE0709F47CC0C63AFDE5F2
:10352000DF0709F481C0C330DD4509F085C080E0C4
:103530006EC080916D0282607DC080916D0216C068
:1035400080916D02886076C080916E0282604FC06B
:1035500080916D0280626EC080916D0280646AC04D
:103560000E941F0780916D02806864C0846062C001
:1035700081603DC080916D028E7F5CC080916D0244
:103580008D7F58C080916D0216C080916E0218C068
:1035900080916E028D7F2BC080916D028F7E4AC01C
:1035A00080916D028F7D46C080916D028F7B42C0FD
:1035B00080916D02877F8B7F3DC080916E028D7FF1
:1035C0008E7F15C080916D0282FB222720F991E049
:1035D000922790FB82F990FB83F92CC080916E02B8
:1035E000982F909591708E7F892B90FB81F9809315
:1035F0006E0222C00E941F0780916D0287FB222766
:1036000020F991E0922790FB87F914C081E00E9495
:10361000F60D12C080916D0284FB222720F991E003
:10362000922790FB84F906C080916D02982F9095A7
:1036300090FB80F980936D0280916D0290916E02F3
:103640000E94770D0E941F0780E001C081E0DF919A
:10365000CF910895CF93DF9386319C4541F5EB01DF
:103660000E94700C982F8A812091020130910301F1
:10367000882379F09A7A81E009F480E080933C0213
:10368000911102C069E201C065E3C9010E94201DD9
:103690000AC080913C02811102C069E201C065E369
:1036A000C9010E942B1D0E94B20C80E001C081E084
:1036B000DF91CF9108950F931F93CF93DF93C42F82
:1036C000D22FFC0182818823C9F040933F020E94DF
:1036D000E31D90933E0280933D0280E28C0F883080
:1036E00008F057C0C77081E001C0880FCA95EAF79B
:1036F000DF91CF911F910F910C947C0480913F0238
:10370000481330C080913D0290913E020E94FB1D03
:10371000883C910538F510E21D0FCD17B9F080E215
:103720008C0F883040F4C77081E001C0880FCA95C3
:10373000EAF70E948304183028F581E09D2F9770E6
:1037400001C0880F9A95EAF70E947C04802F0E949E
:1037500073041830F0F4D77081E001C0880FDA9557
:10376000EAF70AC080E28C0F883098F4C77081E0D5
:1037700001C0880FCA95EAF7DF91CF911F910F9191
:103780000C948304802FDF91CF911F910F910C94A3
:103790007304DF91CF911F910F9108950F939C01B6
:1037A000CB01243F4CE5340731F188F4293DFCE599
:1037B0003F07D9F02A3D4CE5340779F1283D3C45D7
:1037C000A9F506E221EE41EE68ED7CE52BC0263F2F
:1037D000FCE53F07E1F0A8F0273F3C4539F507E25B
:1037E00025EE46EE67EF7CE51DC007E225EE45EECF
:1037F00069ED7CE517C006E221EE40EE64EF7CE562
:1038000011C007E225EE44EE65EF7CE50BC006E251
:1038100021EE42EE66EF7CE505C008E221E045EED0
:103820006AED7CE50E945B1B80E008C0FC018281A0
:10383000882319F010923F0201C081E00F91089592
:1038400090938B0180938A01089590934502809311
:1038500044020895E0914402F0914502309721F02E
:103860000190F081E02D099480E00895E0914402F8
:10387000F0914502309799F020911D01222359F0D3
:1038800020916D0227FF07C0DC012C9111962C932B
:10389000119726E02C930280F381E02D099408957E
:1038A000E0914402F0914502309739F022E0DC01CA
:1038B0002C930480F581E02D099408952091420213
:1038C000309143022817390771F090934302809397
:1038D0004202E0914402F0914502309721F00680C7
:1038E000F781E02D09940895209140023091410222
:1038F0002817390771F09093410280934002E091BC
:103900004402F0914502309721F00084F185E02DCA
:1039100009940895FC01329680911D01882331F0AD
:1039200080916D0287FF02C09EE101C096E080E0B9
:10393000915028F021912223D9F38F5FF9CF089578
:10394000662351F120911D012223E9F020916D029F
:1039500027FF19C0462F4695469546954E31E0F40F
:10396000677021E030E002C0220F331F6A95E2F752
:10397000FC01E40FF11D828190E02823392381E0CE
:10398000232B69F409C0FC01329608962191621735
:1039900029F0E817F907D1F780E0089581E008954C
:1039A0009C01FC0132969FEF80E04191461789F01F
:1039B0009F3F19F4411101C0982F8F5F8630A9F7FE
:1039C0009F3F39F0F901E90FF11D97FDFA956283E8
:1039D000089508959C012A5F3F4FFC0142814613E0
:1039E00001C01282019682179307B9F70895262F16
:1039F0002695269526952E3168F4FC01E20FF11DDF
:103A0000677021E030E001C0220F6A95EAF78281F9
:103A1000282B22830895262F2695269526952E312C
:103A200070F4FC01E20FF11D677021E030E001C08D
:103A3000220F6A95EAF72095828128232283089530
:103A400020911D01222329F020916D0227FD0C9465
:103A5000F71C0C94D01C20911D01222329F02091E9
:103A60006D0227FD0C940B1D0C94EA1C20911D0186
:103A7000FC013296222331F080916D0287FF02C053
:103A80008EE101C086E0DF011D928A95E9F7089575
:103A900008950C94481D83E0809346020C94491DC0
:103AA000811102C081E001C082E0809346020C9443
:103AB000491D0C94501D81E0809346020C94491DD1
:103AC0000C945B1D08950C94621D0C94631D0C9462
:103AD000621D0C94621D0C94621DCF930E94691D9F
:103AE0000E94C5110E94671DC0E08C2F0E94FD102E
:103AF000811104C0CF5FC430C1F701C081E0CF9114
:103B0000089508951F920F920FB60F9211248F936C
:103B10009F93AF93BF9380914702811113C080910F
:103B2000890290918A02A0918B02B0918C024196F9
:103B3000A11DB11D8093890290938A02A0938B02EC
:103B4000B0938C02BF91AF919F918F910F900FBE58
:103B50000F901F90189580919102843031F10E944E
:103B6000CA021092470220E488E190E00FB6F89470
:103B7000A895809360000FBE2093600083B7817F7B
:103B8000846083BF83B7816083BF7894889583B74F
:103B90008E7F83BF0FB6F894A895809160008861EE
:103BA00080936000109260000FBE08950E941F076E
:103BB0000C94D10282E084BD93E095BD9AEF97BD4D
:103BC00080936E0008952FB7F894809189029091A8
:103BD0008A02A0918B02B0918C022FBF08952FB75B
:103BE000F8946091890270918A0280918B02909181
:103BF0008C022FBF08959C014FB7F89480918902E1
:103C000090918A02A0918B02B0918C024FBF821BCF
:103C1000930B089578941F920F920FB60F92112470
:103C20008F939F93AF93BF938091890290918A0263
:103C3000A0918B02B0918C020196A11DB11D8093C1
:103C4000890290938A02A0938B02B0938C02BF9159
:103C5000AF919F918F910F900FBE0F901F9018956D
:103C600087E797E790930108809300089AE088E13E
:103C70000FB6F894A895809360000FBE90936000F3
:103C8000FFCF80916B020895089522E02093E90010
:103C90002FEF3091E800215035FD06C035ED3A9503
:103CA000F1F700002111F5CF2091E80025FF0BC0AE
:103CB00040E050E066E070E00E9484208091E800DF
:103CC0008E778093E8000895CF93DF9320911D01B4
:103CD000222339F020916D0227FF03C060E222E029
:103CE00002C068E021E02093E9002FEF3091E80066
:103CF000215035FD06C035ED3A95F1F70000211150
:103D0000F5CF2091E80025FF1DC0EC0180911D0139
:103D1000811105C040E050E068E070E003C070E051
:103D200040E050E0CE010E9484208091E8008E7730
:103D30008093E80080E2FE01ABE4B2E001900D92D6
:103D40008A95E1F7DF91CF910895809348027093AF
:103D50004A026093490280919102843001F582E029
:103D60008093E9008FEF9091E800815095FD06C0A7
:103D700095ED9A95F1F700008111F5CF8091E8005B
:103D800085FF0DC040E050E063E070E088E492E021
:103D90000E9484208091E8008E778093E800089547
:103DA000BC0184E00C94A51EBC0183E00C94A51E0C
:103DB00080919002811109C00E9415220E947222F6
:103DC0008091E20084608093E20008951092900256
:103DD00008950C94601D60918D0281E0611101C015
:103DE00080E00C944B1D9091910281E0943009F099
:103DF00080E060918D020C94501D42E061EC81E006
:103E00000E948E2142E261EC82E00E948E2190911C
:103E1000910281E0943009F080E060918D020C9471
:103E2000591D80919302833009F461C030F48130D0
:103E300071F0823009F49AC008958A3009F486C07E
:103E40008B3009F46CC0893009F0A8C020C0809183
:103E50009202813A09F0A2C08091E800877F8093A6
:103E6000E8008091960290919702892B21F460E2FC
:103E70008BE492E003C060E080E090E070E00E949C
:103E8000CF208091E8008B778093E800089580919F
:103E90009202813209F082C080919602909197023D
:103EA000029708F07BC08091E800877F8093E8004C
:103EB0008091E80082FD05C0809191028111F8CFC8
:103EC0006DC02091F3008091F20090E0922B029758
:103ED00031F48091F100813011F0863021F480912D
:103EE000F10080936B028091E8008B7753C0809142
:103EF0009202813A09F052C0809196029091970205
:103F0000892B09F04BC08091E800877F8093E800FF
:103F10008091E80080FFFCCF80911D0136C0809128
:103F200092028132D9F58091960290919702892B65
:103F3000A9F58091E800877F8093E8000E94C32163
:103F40008091940280931D010C941F07809192022E
:103F5000813221F58091E800877F8093E8000E94FC
:103F6000C3218091950280936C0208958091920202
:103F7000813AA1F48091E800877F8093E8008091E6
:103F8000E80080FFFCCF80916C028093F10080916B
:103F9000E8008E778093E8000C94C321089584B7DD
:103FA000877F84BF0FB6F894A895809160008861E0
:103FB00080936000109260000FBE90E080E80FB622
:103FC000F89480936100909361000FBE0C945B1D88
:103FD0000E9415220E947222E2EEF0E0808184604D
:103FE000808378940C94072581E191E00C94251C42
:103FF000809191028530A9F480919102853079F405
:104000000E94AB1D80918F028823B1F30E946D1D29
:10401000882391F30E946E200E941F07EDCF0C941D
:10402000D61D089508950C941520292F3327233089
:104030003105C9F060F42130310581F022303105BD
:1040400009F044C08BE390E020E632E043C0213227
:104050003105E1F02232310549F138C082E190E0CA
:104060002BE932E037C099278130910549F028F0DB
:10407000029761F5E8E3F2E005C0ECE5F2E002C08A
:10408000ECE4F2E0849190E09F0124C06115710599
:1040900041F061307105D1F489E090E02BE832E025
:1040A00019C089E090E022E732E014C06115710583
:1040B00041F06130710551F486EB90E02DEA32E079
:1040C00009C080E490E023E633E004C080E090E0A3
:1040D00020E030E0FA0131832083089580E189BD3A
:1040E00082E189BD09B400FEFDCF8091D8008F7DAB
:1040F0008093D8008091E00082608093E0008091FE
:10410000E00081FDFCCF0895CF92DF92EF92FF9205
:104110000F931F93CF93DF93EC018B017A010E94E1
:10412000E221811133C0E114F10439F0F7018081FB
:104130009181081B190BC80FD91FC12CD12C011557
:10414000110519F18091E80085FD16C08091E80005
:104150008E778093E800E114F10449F0F701808143
:104160009181C80ED91ED182C08285E00FC00E9405
:10417000E221882321F30AC089918093F100015044
:104180001109FFEFCF1ADF0ADACF80E0DF91CF917C
:104190001F910F91FF90EF90DF90CF9008952091A5
:1041A0009802309199022617370748F0611571057A
:1041B00039F42091E8002E772093E80001C0B9017E
:1041C000FC0120E06115710579F18091910288234D
:1041D000F1F18530F1F18091E80083FD3CC08091E0
:1041E000E80082FD2EC08091E80080FFEBCF209197
:1041F000F3008091F20090E0922B6115710551F06F
:104200008830910538F421912093F10061507109B3
:104210000196F3CF21E0089709F020E08091E800B3
:104220008E778093E800CECF2111CFCF0AC0809146
:104230009102882361F0853061F08091E80083FD70
:104240000AC08091E80082FFF2CF80E0089582E00A
:10425000089583E0089581E00895209198023091B7
:1042600099022617370748F06115710539F4209136
:10427000E8002E772093E80001C0B901FC0120E09E
:104280006115710591F180919102882309F440C074
:10429000853009F43FC08091E80083FD3DC08091E6
:1042A000E80082FD2FC08091E80080FFE9CF2091D7
:1042B000F3008091F20090E0922B6115710559F0A6
:1042C0008830910540F424912093F100319661509B
:1042D00071090196F2CF21E0089709F020E0809162
:1042E000E8008E778093E800CBCF2111CCCF0AC0B5
:1042F00080919102882361F0853061F08091E8001F
:1043000083FD0AC08091E80082FFF2CF80E008952B
:1043100082E0089583E0089581E00895982F973012
:1043200068F59093E900981739F07091EC002091AE
:10433000ED005091F00003C0242F762F50E021FDB6
:1043400002C09F5FECCF3091EB003E7F3093EB00DB
:104350003091ED003D7F3093ED003091EB00316006
:104360003093EB007093EC002093ED005093F0003D
:104370002091EE0027FDE5CF80E008958F708093B7
:10438000E90081E008958091920287FF11C0809139
:10439000E80082FD05C0809191028111F8CF11C023
:1043A0008091E8008B770BC080919102882349F0BF
:1043B0008091E80080FFF8CF8091E8008E778093AD
:1043C000E80008952091E4003091E50095E64091E1
:1043D000EC00842F817040FF23C08091E80080FDB5
:1043E0001DC080919102882399F0853099F08091C9
:1043F000EB0085FD11C04091E4005091E5002417C9
:10440000350729F3915011F09A01E1CF84E0089526
:1044100082E0089583E0089581E0089580E00895A2
:104420004091E80042FFDDCF08950E9483220E9460
:104430008B22E0EEF0E0808181608083E8EDF0E0A7
:1044400080818F77808319BCA7EDB0E08C918E7F3F
:104450008C9380818F7E80831092900208950F93B9
:104460001F93CF93DF930E9483220E948B22C8ED7B
:10447000D0E088818F77888388818068888388816D
:104480008F7D888319BC1092910210928D02109238
:104490008F0210928E0200EE10E0F80180818B7F77
:1044A000808388818160888342E060E080E00E94B0
:1044B0008E21E1EEF0E080818E7F8083E2EEF0E0FD
:1044C000808181608083808188608083F801808121
:1044D0008E7F8083888180618883DF91CF911F9157
:1044E0000F910895E8EDF0E080818F7E8083E7ED05
:1044F000F0E080818160808384E082BF81E08093EE
:1045000090020C942F22E8EDF0E080818E7F808372
:104510001092E20008951092DA001092E1000895DE
:104520001F920F920FB60F9211242F933F934F9328
:104530005F936F937F938F939F93AF93BF93EF930B
:10454000FF938091E10082FF0BC08091E20082FF27
:1045500007C08091E1008B7F8093E1000E940625D7
:104560008091DA0080FF1FC08091D80080FF1BC0BF
:104570008091DA008E7F8093DA008091D90080FFED
:104580000DC080E189BD82E189BD09B400FEFDCF87
:1045900081E0809391020E94D81E05C019BC109240
:1045A00091020E94E61E8091E10080FF19C0809177
:1045B000E20080FF15C08091E2008E7F8093E200D0
:1045C0008091E20080618093E2008091D800806257
:1045D0008093D80019BC85E0809391020E94EB1E65
:1045E0008091E10084FF30C08091E20084FF2CC004
:1045F00080E189BD82E189BD09B400FEFDCF8091D3
:10460000D8008F7D8093D8008091E1008F7E8093C9
:10461000E1008091E2008F7E8093E2008091E200D1
:1046200081608093E20080918D02882311F084E004
:1046300007C08091E30087FD02C081E001C083E0F4
:10464000809391020E94F31E8091E10083FF29C0B4
:104650008091E20083FF25C08091E100877F8093F5
:10466000E10082E08093910210928D028091E1003E
:104670008E7F8093E1008091E2008E7F8093E20044
:104680008091E20080618093E20042E060E080E09F
:104690000E948E218091F00088608093F0000E943B
:1046A000E91EFF91EF91BF91AF919F918F917F9103
:1046B0006F915F914F913F912F910F900FBE0F908F
:1046C0001F9018951F920F920FB60F9211242F93DF
:1046D0003F934F935F936F937F938F939F93AF938A
:1046E000BF93CF93DF93EF93FF93C091E900CF7017
:1046F0008091EC00D82FD17080FDD0E81092E900B5
:104700008091F000877F8093F00078940E94A62328
:104710001092E9008091F00088608093F000CD2B2A
:10472000CF70C093E900FF91EF91DF91CF91BF91DE
:10473000AF919F918F917F916F915F914F913F9139
:104740002F910F900FBE0F901F9018951F93CF932E
:10475000DF93CDB7DEB7AA970FB6F894DEBF0FBED2
:10476000CDBFE2E9F2E08091F100819322E0EA39E5
:10477000F207C9F70E94111F8091E80083FF2EC144
:104780008091920290919302492F50E04A30510556
:1047900008F024C1FA01EE59FF4F0C947C258038B3
:1047A00021F0823809F01AC108C080918E029091E0
:1047B0008F02992389F082600FC0809196028F70DA
:1047C000873008F00BC18093E9008091EB0085FBF6
:1047D000882780F91092E9009091E800977F9093E4
:1047E000E8008093F1001092F100D1C0282F2D7FB6
:1047F00009F0F4C0882319F0823061F0EFC0809195
:104800009402813009F0EAC0933009F080E080938F
:104810008F022EC08091940281112AC0809196024D
:104820008F702FEF280F263008F0D8C08093E90052
:104830002091EB0020FF1CC0933021F48091EB000D
:10484000806214C09091EB0090619093EB0021E0A6
:1048500030E0A90102C0440F551F8A95E2F740934A
:10486000EA001092EA008091EB0088608093EB00F0
:104870001092E9008091E800877F8093E8000E9411
:10488000C321ACC08111AAC0109194021F778091FE
:10489000E3008078812B8093E3008091E800877F9C
:1048A0008093E8000E94C3218091E80080FFFCCF44
:1048B0008091E30080688093E300111102C082E0E0
:1048C00001C083E08093910289C08058823008F053
:1048D00085C080919402909195028C3D53E095079C
:1048E00079F583E08A838AE289834FB7F894DE0101
:1048F000139620E03EE051E2E32FF0E050935700A2
:10490000E49120FF03C0E295EF703F5FEF708E2FC0
:1049100090E0EA3010F0C79601C0C0968D939D9349
:104920002F5F243149F74FBF8091E800877F809344
:10493000E8006AE270E0CE0101960E94CF2016C026
:104940006091960270919702AE014F5F5F4F0E9497
:104950001320BC01892B09F441C09091E800977F96
:104960009093E80089819A810E942D218091E8002E
:104970008B778093E80032C0803881F58091E80021
:10498000877F8093E80080918D028093F100809171
:10499000E8008E7772CF811121C0809194029091AE
:1049A000950299270297D4F48091E800877F80933D
:1049B000E8008091940280938D020E94C32180912F
:1049C0008D02811106C08091E30087FD02C081E065
:1049D00001C084E0809391020E94FD1E8091E80056
:1049E00083FF0AC08091E800877F8093E800809170
:1049F000EB0080628093EB00AA960FB6F894DEBFBE
:104A00000FBECDBFDF91CF911F9108950895CF9331
:104A1000809191028823A1F0C091E900CF7090911C
:104A2000EC00892F817090FD80E8C82B1092E9007E
:104A30008091E80083FD0E94A623CF70C093E90017
:104A4000CF910895DB018F939F930E949125BF9191
:104A5000AF91A29F800D911DA39F900DB29F900DCD
:104A600011240895AA1BBB1B51E107C0AA1FBB1F3D
:104A7000A617B70710F0A61BB70B881F991F5A95EA
:104A8000A9F780959095BC01CD01089597FB072E5D
:104A900016F4009407D077FD09D00E94322507FC58
:104AA00005D03EF4909581959F4F0895709561953E
:104AB0007F4F0895A1E21A2EAA1BBB1BFD010DC05A
:104AC000AA1FBB1FEE1FFF1FA217B307E407F507BE
:104AD00020F0A21BB30BE40BF50B661F771F881F9A
:104AE000991F1A9469F760957095809590959B0130
:104AF000AC01BD01CF010895EE0FFF1F0590F491A9
:104B0000E02D0994A29FB001B39FC001A39F700D37
:104B1000811D1124911DB29F700D811D1124911DC5
:104B200008950E948225A59F900DB49F900DA49F8B
:104B3000800D911D11240895FB01DC0104C08D91AD
:104B40000190801921F441505040C8F7881B990BFF
:104B50000895F999FECF92BD81BDF89A992780B545
:104B60000895A6E1B0E044E050E00C94E325A8E10C
:104B7000B0E042E050E00C94E325262FF999FECFF7
:104B800092BD81BDF89A019700B4021639F01FBAA0
:104B900020BD0FB6F894FA9AF99A0FBE08950396BD
:104BA000272F0E94BE250E94BD25252F0E94BE25CD
:104BB000242F0C94BE250196272F0E94BE250C940D
:104BC000BD25DC01CB01FC01F999FECF06C0F2BD89
:104BD000E1BDF89A319600B40D9241505040B8F7BB
:064BE0000895F894FFCFD8
:104BE600C800FA01280850011E0A14010004000436
:104BF60004411E641E451ED41ED01E441E01E20042
:104C0600E900EA00B500B600B700CD008301CC008C
:104C16008A0192019401210223022402250226021E
:104C260027022A02B300B4006F007000818283E27B
:104C360000E900EA00B500B600B700CD008301CC5C
:104C4600008A0192019401210223022402250226F0
:104C56000227022A02B300B4006F0070008182832B
:0A4C66009294F6F597C63332000170
:00000001FF
